:020000040000FA
:02000000802856
:02000800E229EB
:100100008B2800308A002108820707340534033425
:100110000234013400348301F901F8010C30A700E6
:10012000A8011830F300F20086018316F030860033
:100130002630870055308100831204309700053047
:100140009D0015309000A921831604308C000130E9
:100150008D0083128C018D018B018B160B178B1771
:100160007810781CB1287810781CB4287810871A79
:10017000BE28F90A871EBA287810B4287C08B10076
:100180007D08B2000310B20CB10C3208A400310893
:10019000A3000310B20CB10C0310B20CB10C310867
:1001A000FA070318FB0A3208FB073108A3070318F4
:1001B000A40A3208A4070310B20CB10C3108FA07E4
:1001C0000318FB0A3208FB070310B20CB10C31080C
:1001D000A3070318A40A3208A4070310B20CB10C39
:1001E0000310B20CB10C3108A3070318A40A32089B
:1001F000A4077A08A5007B08A6007D08B000A1012D
:100200002708A0006C21A200280AF700092903147E
:10021000A20DF70B07299030A9002508B100260888
:10022000B2002308A5070318A60A2408A607812000
:10023000013EF7003008B102031CB203F70B1A2984
:100240003008B1070318B20A3208E039031D2E291D
:100250000F09E039031D2E298F1B2C290F08E039C7
:10026000031D36293209E039031943290F083202E8
:1002700003193D2903182E2943290E0831020319B9
:10028000432903182E290610A21B06140314A20DDD
:10029000220F5129200803193508FF3EA0006C21C8
:1002A000A200A90B20290610A10A2119A11C0029CE
:1002B000B42801308A0021088207FA343C34AD3476
:1002C0002C34C934603420083307F700340803188D
:1002D000013E8A00770882006321F7005921F70761
:1002E000F8100318F814D821F818013E8A0077088E
:1002F000820056344E345334553420344634473417
:10030000483449343B3420344334573451344A342C
:100310005234533420344B3458344C3455345834DC
:10032000493420344C344B34203422344F34553447
:1003300047344C3422342034443448342034543448
:100340005934413445345A345A344E3420342034EC
:100350002034A701A8017930B3000130B400303057
:10036000B500080000000B11F20B0E2A73080319E8
:100370000E2AA803280FD529A70A35082702031932
:10038000A7017708F2000A08F500270864211A3E41
:10039000F70002306721F600A80A0314F60D760F65
:1003A000CC2975088A007208F7007308F2000E2A3B
:1003B00001308A00210882070134033403340434F5
:1003C00002340234FF00030EFE00831203130B19E4
:1003D000B329F90A0C19FD290D1015081B02FC00A0
:1003E0001608031C013E1C02FD00791CF9180E2A98
:1003F0001B08FA001C08FB000D2A0C111B08150233
:10040000FC001C08031C013E1602FD00791CF918B3
:100410000E2A1508FA001608FB0078147E0E8300D9
:10042000FF0E7F0E0900E734E734F734E734F73482
:100430007734773407344F34AF3453344F349734F0
:1004400013344F3447342734AB3423340734073460
:10045000073487346734473467346734C734F73434
:10046000E734F734673467340F3407348F34073494
:100470002F3467346734673467346734EF34EF34CC
:10048000F73467349734EF3497346734EF34FB3400
:10049000F7346734673467346734F7347734773444
:1004A0009734973497347734173467341734673474
:1004B0004F34073417344F344934493449349F3466
:1004C000093449344134093409341F344934493436
:1004D00049340934493409349F3441341F340934D0
:1004E00049341F3409344134F7348F344F341734CE
:1004F000B3343B34973497349734973417341734E4
:1005000007344F34AF34FB34EF3457342B344F348B
:1005100027344734733423340734073407344734DB
:100520009734673497349734A734173417348734A3
:1005300097349734CF3467344F34F7344F3497348B
:1005400097349734973497344F344F341734973463
:1005500097344F34973497344F34AB34173497343F
:1005600097349734973417349734973457349734F3
:10057000973497341734273427344734AF3407344B
:1005800027340F340134013401341F340134013471
:100590000134013401341F34013401340134013495
:1005A000013401341F3401341F34013401341F3449
:1005B0000134013487344F344F3427346B342334BF
:1005C000473467349734F7347734173497347734B3
:1005D000773407344F340F3453346F344734133483
:1005E0000F3427344734FB34FB34073407340734E3
:1005F0004734B73447344734473497347734773403
:100600004734673497340F3407342F3407348F342A
:100610008734D734F734273417344F344F34773492
:100620009734B7344F34B73497344F34AB347734CE
:1006300027342734F7341734773477349734373402
:10064000F7349734973417342734273447340F342A
:10065000073447340F340134493401349F340934AA
:1006600041340934413449349F340134093441342C
:100670004134493441349F3449349F340134413446
:100680001F344934493447342F344F34473403340A
:10069000D334973417341734D73447342734873456
:1006A000F7348734973447349734E73497349734A2
:1006B000173497341734173407344F340F34533406
:1006C000CF342734AB340F342734473473342334D6
:1006D0006734F73407342734D73447342734873422
:1006E000F7348734973447349734E734CF3467345A
:1006F0004F34F7344F344734D734973447341734B2
:100700004F344F3417349734D7344F34D734973469
:100710004F34AB341734473447349734D734173415
:100720009734773437349734973477341734273401
:10073000473447340F34073407340F34013401345D
:1007400001341F34013401340134013401341F34C5
:100750000134013401340134013401341F340134D3
:100760001F34013401341F340134013427344F3431
:100770004F34273403344B34173497344734173409
:1007800097348734973497342734973487349734A1
:100790009734973497341734173407340F340F34A1
:1007A000FB34EF34A7344B340F3427344734AB34A5
:1007B00023344734073467342734973447341734A5
:1007C0009734873497349734273497348734CF3429
:1007D00047348F3407342F34073417349734973421
:1007E00097344F344F341734973497344F34973409
:1007F00097344F348B341734973497349734973475
:100800001734973417345734973497345734173490
:100810002734473447340F34073407340F3409344E
:10082000013401341F3449340934013401340134B2
:100830009F344934013449340934093449349F34EC
:1008400041341F34493401349F340934013417349E
:100850004F344F3427340334C3345734E7347734B8
:100860009734773477343734773497348734673430
:1008700077346734E734073467344734F734673400
:100880008734673467342734673487349734773450
:1008900067347734F734173407344F340F34533414
:1008A0004F349734B3340F3447342734033403348C
:1008B000273407346734173467344734F7346734E0
:1008C0008734673467342734673487340F342734E8
:1008D0000F3407340F344734E734973467346734C0
:1008E000EF34EF341734673497344F349734673428
:1008F0004F348B34F7346734673497346734F734C4
:10090000773417349734973467349734F73467342F
:10091000873467340F34F73407340F34013401342B
:1009200001341F34013401340134013401341F34E3
:100930000134013401340134013401341F340134F1
:100940001F34013401341F3401340134F7348F343F
:080950004F3417340334433423
:00000001FF
